:100000003EC10000BEC7000093C7000068C70000E3
:100010003DC7000012C70000E7C6000060C1000035
:100020005EC100005CC100005AC1000058C1000060
:1000300056C1000054C1000052C1000050C1000070
:100040004EC100004CC100004AC1000048C1000080
:1000500046C1000044C1000042C100007BC6000050
:100060003EC1000041C6000016C6000038C10000B5
:1000700036C1000034C1000032C1000030C10000B0
:100080002EC100002CC100002AC1000028C10000C0
:1000900026C1000024C1000022C1000020C10000D0
:1000A0001EC100001CC100001AC1000018C10000E0
:1000B00016C1000014C1000012C1000010C10000F0
:1000C0000EC100000CC100000AC1000008C1000000
:1000D00006C1000004C1000002C1000000C1000010
:1000E000FEC000002F0A002300230023005C23230E
:1000F00023235265616C53696D476561722300006B
:100100000020002300260029002C002F00320000D0
:10011000010000030106010901000021002400275D
:10012000002A002D00300033000101000004010707
:10013000010A0100002200250028002B002E0031BA
:1001400000340002010000050108010B010505054E
:1001500005070508080808020202020A0A0808043E
:10016000040404010101010101010103030303036C
:10017000030303040707070C0C0C0C0C0C0C0C02FB
:1001800002020206060606060606060B0B0B0B0B02
:100190000B0B0B01021020200808102040102040FB
:1001A000800201020108040201010204081020403B
:1001B0008080402010080402018004020180402059
:1001C0001008040201080402010102040810204082
:1001D00080010204081020408000000A0B02090C74
:1001E0000D0E0807030401000000000000000000DD
:1001F00000000000000000000000000000000000FF
:1002000000000000001211100000000000000000BB
:100210000000000000000000000000000000002FAF
:100220000A002300230023005C232323235265615B
:100230006C53696D4765617223000A000A003D0036
:100240000A003D003D300A002E4F46460A003D316F
:100250000A002E4F4E0A003D300A003D310A002FA1
:100260000A002300230023005C232323235265611B
:100270006C53696D476561722300EA076E0B1124A8
:100280001FBECFEFD1E2DEBFCDBF00E00CBF27E045
:10029000A8E3B4E001C01D92A536B207E1F714E06F
:1002A000A0E0B2E0E0E1FCE100E00BBF02C007909B
:1002B0000D92A833B107D9F711E0CEE3D1E000E009
:1002C00006C021970109802FFE010E94BC0BCD338F
:1002D000D10780E00807A9F718D70C94F70D90CE46
:1002E000AF92BF92CF92DF92EF92FF920F931F9344
:1002F000CF93DF936C017B018B01040F151FEB0182
:100300005E01AE18BF08C017D10759F06991D60138
:10031000ED91FC910190F081E02DC6011995892B9A
:1003200079F7C501DF91CF911F910F91FF90EF9069
:10033000DF90CF90BF90AF900895E1E5F5E0448164
:100340005581608171818BEA94E0CACFFC01538DA5
:10035000448D252F30E0842F90E0821B930B54179F
:1003600010F0CF96089501970895FC01918D828D2C
:10037000981761F0A28DAE0FBF2FB11D5D968C91C5
:10038000928D9F5F9F73928F90E008958FEF9FEF04
:100390000895FC01918D828D981731F0828DE80FC0
:1003A000F11D858D90E008958FEF9FEF0895FC017A
:1003B000918D228D892F90E0805C9F4F821B910947
:1003C0008F73992708958BEA94E0F1DF21E0892B60
:1003D00009F420E0822F0895FC01A48DA80FB92F05
:1003E000B11DA35ABF4F2C91848D90E001968F735D
:1003F0009927848FA689B7892C93A089B1898C917C
:10040000837080648C93938D848D981306C00288CA
:10041000F389E02D80818F7D80830895EF92FF9294
:100420000F931F93CF93DF93EC0181E0888F9B8D17
:100430008C8D98131AC0E889F989808185FF15C0D1
:100440009FB7F894EE89FF896083E889F9898081F4
:100450008370806480839FBF81E090E0DF91CF91C3
:100460001F910F91FF90EF900895F62E0B8D10E0E5
:100470000F5F1F4F0F731127E02E8C8D8E110BC055
:100480000FB607FCFACFE889F989808185FFF5CF9F
:10049000CE01A2DFF2CFEB8DEC0FFD2FF11DE35A61
:1004A000FF4FF0829FB7F8940B8FEA89FB89808118
:1004B0008062D0CF0F931F93CF93DF938C01D0E056
:1004C000C0E0F801EC0FFD1F6491662339F08BEA60
:1004D00094E0A4DF892B11F02196F3CFCE01DF91B8
:1004E000CF911F910F910895CF93DF93EC01888DE9
:1004F0008823B1F0AA89BB89E889F9898C9185FDA7
:1005000003C0808186FD0CC00FB607FCF7CF8C912D
:1005100085FFF2CF808185FFEDCFCE015DDFEACF91
:10052000DF91CF9108958150823108F05AC0E82FB1
:10053000F0E08827E156FD4F8F4F0C94BC0BBF02B3
:10054000C302B102B702BB02F102C602CC02D00262
:10055000D602DA02DE02E402E802F102EC02F20262
:10056000F602809180008F778093800008958091BB
:1005700080008F7DF9CF80918000877FF5CF84B593
:100580008F7784BD089584B58F7DFBCF8091B000B7
:100590008F778093B00008958091B0008F7DF9CF60
:1005A000809190008F7780939000089580919000C3
:1005B0008F7DF9CF80919000877FF5CF8091A0004B
:1005C0008F778093A00008958091A0008F7DF9CF50
:1005D0008091A000877FF5CF809120018F77809355
:1005E00020010895809120018F7DF9CF8091200115
:1005F000877FF5CF1F93CF93DF93282F30E0F9014A
:10060000E752FE4F8491F901ED56FE4FD491F90166
:10061000E35BFE4FC491CC23A1F0162F811183DF41
:10062000EC2FF0E0EE0FFF1FED5CFE4FA591B491B3
:100630008FB7F894EC91111108C0D095DE23DC93AC
:100640008FBFDF91CF911F910895DE2BF8CFCF930D
:10065000DF9390E0FC01ED56FE4F2491835B9E4FAB
:10066000FC0184918823C9F090E0880F991FFC0158
:10067000E75EFE4FA591B491FC01ED5CFE4FC59184
:10068000D49161110DC09FB7F8948C91209582236D
:100690008C938881282328839FBFDF91CF91089571
:1006A000623051F49FB7F8943C91822F8095832358
:1006B0008C93E8812E2BEFCF8FB7F894EC912E2BF3
:1006C0002C938FBFEACF862F642FC1CF863308F0DB
:1006D000865320917B00982F9870277F922B9093C0
:1006E0007B008770806480937C0080917A008064B6
:1006F00080937A0080917A0086FDFCCF809178000B
:100700009091790008953FB7F8948091A304909157
:10071000A404A091A504B091A60426B5A89B05C089
:100720002F3F19F00196A11DB11D3FBFBA2FA92F70
:10073000982F8827BC01CD01620F711D811D911D6D
:1007400042E0660F771F881F991F4A95D1F70895D9
:100750008F929F92AF92BF92CF92DF92EF92FF92D1
:100760004B015C01D0DF6B017C01CDDF6C197D0991
:100770008E099F09683E734081059105B0F321E021
:10078000821A9108A108B10888EEC80E83E0D81E2D
:10079000E11CF11C81149104A104B10431F7FF9014
:1007A000EF90DF90CF90BF90AF909F908F90089583
:1007B0002FB7F89460919F047091A0048091A104D8
:1007C0009091A2042FBF0895FC01808580FD04C094
:1007D00082FB882780F9089580E00895FC019085C8
:1007E000957081E0953009F080E00895CF92DF9216
:1007F000EF92FF920F931F93CF93DF93EC018885C5
:100800008B7F8887E881F9810190F081E02DCE010E
:100810001995182F8885869581701817B1F0C8DF53
:100820006A837B838C839D83888592E08927888770
:10083000888582FB882780F9DF91CF911F910F91E6
:10084000FF90EF90DF90CF900895B2DFCA80DB80F9
:10085000EC80FD80AB01BC014C195D096E097F097C
:100860008E819F81B0E0A0E0481759076A077B0797
:10087000F8F2888581701817D9F29ADF6A837B8332
:100880008C839D83888591E089278460888790DFA9
:100890000A851B852C853D85601B710B820B930B94
:1008A0006E877F87888B998B83DF6A877B878C87AE
:1008B0009D87BECFCF93DF93EC0169871886E881CF
:1008C000F9810190F081E02D1995882319F0888530
:1008D000836088876DDF6A837B838C839D83DF9150
:1008E000CF910895CF93DF93FC01218530E0F9018A
:1008F000E752FE4F8491F901ED56FE4FD491F90174
:10090000E35BFE4FC491CC2371F081110CDEEC2F20
:10091000F0E0EE0FFF1FE150FF4FA591B491EC9175
:10092000ED2381E009F480E08170DF91CF9108959B
:10093000DC01ED91FD918081ED91FD919081ED9132
:10094000FD916C9163708E2309F064609F2309F020
:100950006860E5EBF4E0E60FF11D659565956D9334
:100960006D917D918D919D91099423C01AC012C003
:1009700016C010C01EC009C014C013C006C019C0E4
:1009800009C00DC007C00DC014C062507040804047
:1009900090400BC0615070408040904006C06E5F38
:1009A00001C06F5F7F4F8F4F9F4F9E938E937E93BB
:1009B0006E9308958F929F92AF92BF920F931F9361
:1009C000CF93DF93CDB7DEB7A1970FB6F894DEBF14
:1009D0000FBECDBF19A2423008F44AE08E010F5D70
:1009E0001F4F842E912CB12CA12CA5019401A2D6CD
:1009F000E62FB901CA01EA303CF5E05DD801EE937B
:100A00008D01232B242B252B81F790E080E010977C
:100A100061F0FD0101900020E9F73197AF014A1B19
:100A20005B0BBD018BEA94E05BDCA1960FB6F894FA
:100A3000DEBF0FBECDBFDF91CF911F910F91BF9051
:100A4000AF909F908F900895E95CD8CFCF92DF92BE
:100A5000EF92FF92CF93DF936C01990FEE08FF089E
:100A6000F7FE17C06DE28BEA94E0D8DCEC01662754
:100A70007727CB016C197D098E099F094AE09ADF1F
:100A80008C0F9D1FDF91CF91FF90EF90DF90CF9063
:100A900008954AE0C701B601DF91CF91FF90EF9032
:100AA000DF90CF9087CF009761F0FC01019000208C
:100AB000E9F73197AF01481B590BBC018BEA94E071
:100AC0000FCC90E080E008950F931F93CF93DF93B6
:100AD0008BEA94E06CDC892B09F450C08BEA94E03B
:100AE00044DC8C37D1F48DEE90E0E4DC84EA92E0D3
:100AF000DADF8BEE90E0DEDC86E090E0A7DF89EEC7
:100B000090E0D8DC84E092E0CEDF87EE90E0D2DCAB
:100B100014DC84EE90E0CEDCDBCF8C3329F4109231
:100B20009D0410929C04D4CF8A30B1F4C4E1D2E089
:100B300008E314E089919991009739F0F801208138
:100B400061E0213309F060E055DD0F5F1F4FF2E0F7
:100B5000CA31DF0779F7E3CF20919C0430919D04DF
:100B600024363105E4F6F901E85CFB4F80832F5F02
:100B70003F4F30939D0420939C04AACFDF91CF91E7
:100B80001F910F9108951FDC81119EDF80E090E09E
:100B9000892B49F080E090E0892B29F00E94000029
:100BA00081110E94000080E090E0892B49F080E0F4
:100BB00090E0892B29F00E94000081110E94000022
:100BC00080E090E0892B49F080E090E0892B29F0CB
:100BD0000E94000081110C9400000895CF93DF93D0
:100BE000EC0188819981009709F06AD619821882F0
:100BF0001D821C821B821A82DF91CF910895FC0115
:100C000080819181009709F05BC608950F931F932F
:100C1000CF93DF93EC0188819981009759F02A8165
:100C20003B812617370730F081E0DF91CF911F918C
:100C30000F9108958B016F5F7F4FCBD6009759F0CE
:100C4000998388831B830A832C813D81232B61F741
:100C5000FC011082E9CF80E0E8CFEF92FF920F9382
:100C60001F93CF93DF93EC017B018A01BA01CEDFA2
:100C700081110AC0CE01B2DFCE01DF91CF911F9169
:100C80000F91FF90EF9008951D830C83B701888129
:100C900099818CD7F1CF1F920F920FB60F9211242A
:100CA0000BB60F922F933F934F935F936F937F9366
:100CB0008F939F93AF93BF93EF93FF938BEA94E04F
:100CC0008BDBFF91EF91BF91AF919F918F917F91BE
:100CD0006F915F914F913F912F910F900BBE0F90AD
:100CE0000FBE0F901F9018951F920F920FB60F9284
:100CF00011240BB60F922F938F939F93EF93FF9333
:100D0000E091BB04F091BC048081E091C104F091BA
:100D1000C20482FD1DC090818091C4048F5F8F73D7
:100D20002091C504821741F0E091C404F0E0E5553C
:100D3000FB4F958F8093C404FF91EF919F918F910A
:100D40002F910F900BBE0F900FBE0F901F90189514
:100D50008081F2CF1F920F920FB60F9211242F9322
:100D60003F938F939F93AF93BF9380919F049091F4
:100D7000A004A091A104B091A20430919E0423E0AC
:100D8000230F2D3758F50196A11DB11D20939E0408
:100D900080939F049093A004A093A104B093A20415
:100DA0008091A3049091A404A091A504B091A604FD
:100DB0000196A11DB11D8093A3049093A404A09358
:100DC000A504B093A604BF91AF919F918F913F91DD
:100DD0002F910F900FBE0F901F90189526E8230FAC
:100DE0000296A11DB11DD2CF1F920F920FB60F9286
:100DF00011240BB60F922F933F934F935F936F93F2
:100E00007F938F939F93AF93BF93EF93FF9390E064
:100E100080E08EDDFF91EF91BF91AF919F918F9117
:100E20007F916F915F914F913F912F910F900BBEEA
:100E30000F900FBE0F901F9018951F920F920FB634
:100E40000F9211240BB60F922F933F934F935F9302
:100E50006F937F938F939F93AF93BF93EF93FF9382
:100E600090E080E065DDFF91EF91BF91AF919F91A0
:100E70008F917F916F915F914F913F912F910F9043
:100E80000BBE0F900FBE0F901F9018951F920F92E0
:100E90000FB60F9211240BB60F922F933F934F93DF
:100EA0005F936F937F938F939F93AF93BF93EF93D2
:100EB000FF9390E080E03CDDFF91EF91BF91AF9117
:100EC0009F918F917F916F915F914F913F912F9162
:100ED0000F900BBE0F900FBE0F901F9018951F9292
:100EE0000F920FB60F9211240BB60F922F933F93D0
:100EF0004F935F936F937F938F939F93AF93BF9322
:100F0000EF93FF9390E080E013DDFF91EF91BF91AD
:100F1000AF919F918F917F916F915F914F913F9191
:100F20002F910F900BBE0F900FBE0F901F90189532
:100F30001F920F920FB60F9211240BB60F922F93A0
:100F40003F934F935F936F937F938F939F93AF9351
:100F5000BF93EF93FF9390E080E0EADCFF91EF9185
:100F6000BF91AF919F918F917F916F915F914F91C1
:100F70003F912F910F900BBE0F900FBE0F901F90BF
:100F800018951F920F920FB60F9211240BB60F9265
:100F90002F933F934F935F936F937F938F939F9381
:100FA000AF93BF93EF93FF9390E080E0C1DCFF919C
:100FB000EF91BF91AF919F918F917F916F915F91D1
:100FC0004F913F912F910F900BBE0F900FBE0F903E
:100FD0001F9018951092AE041092AD0488EE93E025
:100FE000A0E0B0E08093AF049093B004A093B1046C
:100FF000B093B2048EE892E09093AC048093AB047B
:1010000085EC90E09093B8048093B70484EC90E072
:101010009093BA048093B90480EC90E09093BC0460
:101020008093BB0481EC90E09093BE048093BD0458
:1010300082EC90E09093C0048093BF0486EC90E033
:101040009093C2048093C1041092C4041092C5040A
:101050001092C6041092C704A8E4B5E090E080E0C6
:1010600041E2FC013E9621E030E08630910510F42B
:1010700030E020E0E20FF31F40935700E491ED933E
:1010800001968930910569F780EA92E090935007C4
:1010900080934F07109251071092520710925307F6
:1010A000109254078AE090E090935607809355077A
:1010B0001092570710925807E7E5F5E08FE497E0A4
:1010C00040EA52E02AE030E05183408312821382EA
:1010D00014821582378326831086118672968E17A6
:1010E0009F0791F7109252051092510510925405E6
:1010F00010925305109256051092550550E040E0AD
:101100006EEC72E081E595E0A8CDCF93DF93CDB78B
:10111000DEB72F970FB6F894DEBF0FBECDBF789421
:1011200084B5826084BD84B5816084BD85B58260EC
:1011300085BD85B5816085BD80916E00816080939D
:101140006E00109281008091810082608093810006
:101150008091810081608093810080918000816016
:10116000809380008091B10084608093B100809171
:10117000B00081608093B000809191008260809384
:101180009100809191008160809391008091900006
:101190008160809390008091A10082608093A10083
:1011A0008091A10081608093A1008091A000816066
:1011B0008093A00080912101826080932101809121
:1011C00021018160809321018091200181608093C1
:1011D000200180917A00846080937A0080917A0067
:1011E000826080937A0080917A00816080937A0097
:1011F00080917A00806880937A001092C100E0911B
:10120000BB04F091BC0482E08083E091B704F091CC
:10121000B8041082E091B904F091BA0480E18083AF
:101220001092C304E091BF04F091C00486E0808373
:10123000E091BD04F091BE04808180618083E091E3
:10124000BD04F091BE04808188608083E091BD047C
:10125000F091BE04808180688083E091BD04F091AC
:10126000BE0480818F7D808382E390E0A0E0B0E0C7
:101270008093AF049093B004A093B104B093B204F0
:1012800068EE73E080E090E063DA69E4C62E65E022
:10129000D62E8E010F5F1F4FD6018D916D011B86DB
:1012A0001A861D861C861F861E8640E1B80190E0C6
:1012B00018D2F80101900020E9F73197AF01401BE7
:1012C000510BB801CE010A96C8DC1A8219821C8221
:1012D0001B821E821D82609151057091520561151D
:1012E000710531F04091550550915605C801B5DCA6
:1012F0008E859F85AA84BB84ED80FE80E80EF91E52
:10130000A114B10409F439C0892B79F0B701C801DF
:101310007DDC882391F129813A818D819E81B501FF
:10132000820F931F43D4FE82ED8269817A81611519
:10133000710531F14D815E8181E595E08EDCC8015A
:101340005EDCCE010A965BDCB1E5CB16B5E0DB06D0
:1013500009F0A2CF00915105109152050115110518
:1013600099F0F8018081882379F0082E000C990B00
:101370000CD4D8018D938D01F4CFC8012FDCD5CFCB
:1013800081E595E02BDCDBCF88E292E093D884EA1C
:1013900092E089DB86E292E08DD886E090E056DB31
:1013A00084E292E087D884E092E07DDB82E292E002
:1013B00081D80E949D018FE192E07CD862E08AE1B1
:1013C00046D96AE170E08FE497E074DA8AE090E051
:1013D000909356078093550707E515E04AE1E42E00
:1013E00042E0F42E5AE0A52EB12CF701C080D18046
:1013F000D801ED91FC910280F381E02D42E050E0B4
:10140000B601C8011995B601C80154DAF801B782CE
:10141000A682F4E0EF0EF11C0E5E1F4F87E00F3442
:10142000180719F724E1E22E22E0F22E3AE1A32E6A
:1014300032E0B32ED701CD90DD907D01C114D104EF
:1014400031F061E08C2D03D961E08C2DD3D8AE143E
:10145000BF0481F768EB7BE080E090E079D960E041
:101460008EE2C8D860E08FE2C5D860E080E3C2D8E1
:101470009FD96B017C0180910A0290910B02A0918F
:101480000C02B0910D02AC01BD014854544F6F4F96
:101490007F4FC416D506E606F70628F4C816D90607
:1014A000EA06FB0670F588E692E004D884EA92E04A
:1014B000FADA86E692E00E945A0286E090E0C6DA06
:1014C00084E692E00E945A0284E092E0ECDA82E63E
:1014D00092E00E945A020E949D018FE592E00E94D4
:1014E0005A02C0920A02D0920B02E0920C02F092D1
:1014F0000D02C0920002D0920102E0920202F0922C
:1015000003028FE497E072D98FE497E05DD98111EF
:1015100005C08FE497E062D98823D1F08BEB92E08D
:10152000C2DA8FE497E050D9882309F4B0C08BE584
:1015300092E00E945A0264E670E080E090E008D9F0
:10154000C0920002D0920102E0920202F0920302E5
:1015500061E070E080E090E0FBD88AE1682E82E0F4
:10156000782E97E5A92E95E0B92EC5013FD9C50182
:101570002BD9882309F499C0F301828093806AE112
:1015800074E0C4011AD3892B09F48AC0C4018BDA30
:1015900082E592E00E945A02B2E1AB0EB11CE4E097
:1015A0006E0E711C0A151B0501F786E38FD85C01CE
:1015B0008091A9049091AA049C012F503109A21690
:1015C000B30624F00F968A159B05ACF4FBE0AF162A
:1015D000B1048CF0B092AA04A092A90483EC92E02A
:1015E00062DA82E492E00E945A02C5012FDA80E4B6
:1015F00092E00E945A0287E369D85C018091A704B7
:101600009091A8049C012F503109A216B30624F032
:101610000F968A159B05ACF48BE0A816B1048CF0EC
:10162000B092A804A092A7048FEC92E03CDA8EE37B
:1016300092E00E945A02C50109DA8CE392E00E940E
:101640005A028091000290910102A0910202B09191
:101650000302AC01BD014C595F4F6F4F7F4FC41661
:10166000D506E606F70628F4C816D906EA06FB06EC
:1016700060F48AE392E00E945A02C0920002D09283
:101680000102E0920202F09203027DDAF1CE8FE4D1
:1016900097E0A4D8882309F44ECF87E592E049CF9C
:1016A000C40101DA8EE492E075CFC50197D8882392
:1016B00009F472CFD30112968D909C906AE174E088
:1016C000C4017BD2892B29F0C401EDD988E492E0D2
:1016D00061CFC401E8D984E492E05CCF81E595E074
:1016E0008ECABB27FB015527AA27880F991FAA1F5F
:1016F000A41710F0A41B83955051B9F7A05DAA332D
:1017000008F0A95DA193009779F7B111B1931192F7
:10171000CB0100C0DC01FC01672F71917723E1F759
:10172000329704C07C916D9370836291AE17BF07AE
:10173000C8F30895A1E21A2EAA1BBB1BFD010DC020
:10174000AA1FBB1FEE1FFF1FA217B307E407F50771
:1017500020F0A21BB30BE40BF50B661F771F881F4D
:10176000991F1A9469F760957095809590959B01E3
:10177000AC01BD01CF010895EE0FFF1F881F8BBF85
:101780000790F691E02D19940F931F93CF93DF9359
:101790008230910510F482E090E0E0916307F091CF
:1017A000640730E020E0B0E0A0E0309799F4211524
:1017B000310509F44AC0281B390B24303105D8F50E
:1017C0008A819B816115710589F1FB019383828375
:1017D000FE0111C0408151810281138148175907D0
:1017E000E0F04817590799F4109761F012960C939E
:1017F000129713961C933296CF01DF91CF911F91D0
:101800000F9108950093630710936407F4CF211597
:10181000310551F04217530738F0A901DB019A0155
:10182000BD01DF01F801C1CFEF01F9CF909364074B
:1018300080936307CDCFFE01E20FF31F8193919355
:101840002250310939832883D7CF20916107309105
:101850006207232B41F42091100230911102309342
:1018600062072093610720910E0230910F0221152B
:10187000310541F42DB73EB7409112025091130249
:10188000241B350BE0916107F0916207E217F30723
:10189000A0F42E1B3F0B2817390778F0AC014E5FE0
:1018A0005F4F2417350748F04E0F5F1F50936207B4
:1018B00040936107819391939FCFF0E0E0E09CCF4C
:1018C000CF93DF930097E9F0FC01329713821282E5
:1018D000A0916307B0916407ED0130E020E010971C
:1018E000A1F420813181820F931F209161073091F3
:1018F00062072817390709F061C0F0936207E09387
:101900006107DF91CF910895EA01CE17DF07E8F56F
:101910004A815B819E0141155105B1F7E901FB83C5
:10192000EA8349915991C40FD51FEC17FD0761F463
:10193000808191810296840F951FE90199838883A4
:10194000828193819B838A83F0E0E0E012968D91FF
:101950009C9113970097B9F52D913C911197CD016A
:101960000296820F931F209161073091620728171A
:10197000390739F6309751F51092640710926307D2
:10198000B0936207A0936107BCCFD383C283408129
:101990005181840F951FC817D90761F44E5F5F4FBF
:1019A00088819981480F591F518340838A819B8187
:1019B000938382832115310509F0B0CFF09364073A
:1019C000E09363079ECFFD01DC01C0CF138212823A
:1019D000D7CF4F925F926F927F928F929F92AF92EA
:1019E000BF92CF92DF92EF92FF920F931F93CF930C
:1019F000DF938C01009791F4CB01DF91CF911F9180
:101A00000F91FF90EF90DF90CF90BF90AF909F909D
:101A10008F907F906F905F904F90B6CEFC01E60F55
:101A2000F71F9C0122503109E217F30708F4AAC0FE
:101A3000D901CD91DC911197C617D70718F1C530A0
:101A4000D10570F0CE0104978617970748F0C61BA2
:101A5000D70B2297C193D1936D937C93CF0130DF45
:101A6000C801DF91CF911F910F91FF90EF90DF9010
:101A7000CF90BF90AF909F908F907F906F905F902E
:101A80004F9008955B01AC1ABD0A4C018C0E9D1E4F
:101A9000A0916307B0916407512C412CF12CE12CEB
:101AA000109731F58091610790916207881599052B
:101AB00009F05CC04616570608F058C080910E0227
:101AC00090910F02009741F48DB79EB7409112029A
:101AD00050911302841B950BE817F90708F052C0C8
:101AE000F0936207E0936107F90171836083B8CFD7
:101AF0008D919C91119712966C90129713967C90F1
:101B00001397A815B90559F56C0142E0C40ED11C14
:101B1000CA14DB0420F1AC014A195B09DA01129600
:101B2000159780F06282738251834083D9016D934F
:101B30007C93E114F10471F0D7011396FC93EE93BA
:101B400012978ECF22968C0F9D1FF901918380836F
:101B5000F301EFCFF0936407E093630781CF48165A
:101B6000590608F42C017D01D3019ACFCB010CDE7C
:101B70007C01009739F0AE01B8010FD0C801A0DE9A
:101B800087016ECF10E000E06BCF91110895815670
:101B90008A5108F4805285580895FB01DC0102C087
:101BA00001900D9241505040D8F70895FB01DC019F
:101BB00001900D920020E1F70895FB01519155230A
:101BC000A9F0BF01DC014D9145174111E1F759F42E
:101BD000CD010190002049F04D9140154111C9F30C
:101BE000FB014111EFCF81E090E00197089511E0F2
:101BF000CEE3D1E000E005C0802FFE01BDDD2196DF
:101C0000011DCF33D10780E00807B1F7F894FFCF6B
:101C1000FFFFFFFF332E312E3900FFFFFFFF0000D3
:101C2000650780002E002F0030001D00DB0227001A
:101C3000E7020E00F3020F00FE021E0009031F0060
:101C400018032000220321002F0322003903230060
:101C50004903240055032500610328006F03290070
:101C60007E03160088031700930318009E031900D3
:101C7000A9031A00B4032A00BF031500CF032D00E7
:101C8000E0031400EC031300F8032C00040412001A
:101C9000100426001E042B002B04000000000E027E
:101CA0007001A6017402D701B501C901000000004E
:101CB000720463035265616C53696D476561722DEF
:101CC0004349525255532D5357310053575F4B459B
:101CD000593500504F545F44494D4D4552310050E5
:101CE0004F545F44494D4D4552320053575F424176
:101CF0005454322E53570053575F42415454312E9F
:101D000053570053575F414C54312E53570053578C
:101D10005F414C54322E53570053575F4156494F41
:101D20004E4943532E53570053575F4E41562E533F
:101D3000570053572E5354524F42452E535700537A
:101D4000575F4C44472E53570053575F4943455FF5
:101D50004C494748542E53570053575F5049544FEE
:101D6000542E53570053575F4943494E472E5357FC
:101D70000053575F4943455F4C564C2E5357005311
:101D8000575F4943455F50554D502E5357005357A9
:101D90005F5331342E53570053575F4B4559312E03
:101DA00053570053575F4B4559322E5357005357E3
:101DB0005F4B4559332E53570053575F4B455934AA
:101DC0002E53570053575F4B4559352E53570053E9
:101DD000575F4655454C5F50554D502E5357005355
:101DE000575F4655454C5F5052494D452E5357005D
:101DF00053575F4655454C312E53570053575F4656
:101E000055454C322E53570053575F4655454C337A
:101E10002E53570053575F4655454C342E535700A9
:101E200053572E464C41503130302E5357005357A4
:101E30005F464C415035302E53570053575F464C48
:081E40004150302E5357000001
:00000001FF
